Home Database Mysql Tutorial Oracle的数据表压缩

Oracle的数据表压缩

Jun 07, 2016 pm 05:33 PM
database

Oracle的数据表压缩,压缩原理:将同一个Block里所有行的重复列值存储在表头的一块区域。该块区域被称为符号表(symbol table)。

Oracle的数据表压缩
压缩原理:将同一个Block里所有行的重复列值存储在表头的一块区域。该块区域被称为符号表(symbol table)。行里如果有某列的值等于
符号表里存储的值,则不存储实际的值,只存储该值在符号表里的地址。

表压缩技术适合的对象:
Block里含有重复列值的数据表;
读取较多,更改较少的表。

数据表压缩的优点:
对于Block里含有重复列值的数据表,可以极大的节省存储空间,并减少IO和占用的内存。
数据表压缩的缺点:
CPU需要进行压缩和解压操作,存在额外的消耗。
DBA需对数据的分布有一个较好的认识。

CREATE TABLE a
(a NUMBER(5),
b VARCHAR2(30) )
COMPRESS;


CREATE TABLE b
(a NUMBER(5),
b VARCHAR2(30) );

insert into a values(1,'aaaaaaaaaaaaaaaa');
insert into a values(2,'aaaaaaaaaaaaaaaa');
insert into a values(3,'aaaaaaaaaaaaaaaa');


insert into b values(1,'aaaaaaaaaaaaaaaa');
insert into b values(2,'aaaaaaaaaaaaaaaa');
insert into b values(3,'aaaaaaaaaaaaaaaa');


data_block_dump,data header at 0x2b3b07180264
===============
tsiz: 0x1f98
hsiz: 0x18
pbl: 0x2b3b07180264
76543210
flag=--------
ntab=1
nrow=3
frre=-1
fsbo=0x18
fseo=0x1f53
avsp=0x1f3b
tosp=0x1f3b
0xe:pti[0] nrow=3 offs=0
0x12:pri[0] offs=0x1f81
0x14:pri[1] offs=0x1f6a
0x16:pri[2] offs=0x1f53
block_row_dump:
tab 0, row 0, @0x1f81
tl: 23 fb: --H-FL-- lb: 0x1 cc: 2
col 0: [ 2] c1 02
col 1: [16] 61 61 61 61 61 61 61 61 61 61 61 61 61 61 61 61
tab 0, row 1, @0x1f6a
tl: 23 fb: --H-FL-- lb: 0x1 cc: 2
col 0: [ 2] c1 03
col 1: [16] 61 61 61 61 61 61 61 61 61 61 61 61 61 61 61 61
tab 0, row 2, @0x1f53
tl: 23 fb: --H-FL-- lb: 0x1 cc: 2
col 0: [ 2] c1 04
col 1: [16] 61 61 61 61 61 61 61 61 61 61 61 61 61 61 61 61
end_of_block_dump
Block dump from cache:

data_block_dump,data header at 0xf427c064
===============
tsiz: 0x1f98
hsiz: 0x18
pbl: 0xf427c064
76543210
flag=--------
ntab=1
nrow=3
frre=-1
fsbo=0x18
fseo=0x1f53
avsp=0x1f3b
tosp=0x1f3b
0xe:pti[0] nrow=3 offs=0
0x12:pri[0] offs=0x1f81
0x14:pri[1] offs=0x1f6a
0x16:pri[2] offs=0x1f53
block_row_dump:
tab 0, row 0, @0x1f81
tl: 23 fb: --H-FL-- lb: 0x1 cc: 2
col 0: [ 2] c1 02
col 1: [16] 61 61 61 61 61 61 61 61 61 61 61 61 61 61 61 61
tab 0, row 1, @0x1f6a
tl: 23 fb: --H-FL-- lb: 0x1 cc: 2
col 0: [ 2] c1 03
col 1: [16] 61 61 61 61 61 61 61 61 61 61 61 61 61 61 61 61
tab 0, row 2, @0x1f53
tl: 23 fb: --H-FL-- lb: 0x1 cc: 2
col 0: [ 2] c1 04
col 1: [16] 61 61 61 61 61 61 61 61 61 61 61 61 61 61 61 61
end_of_block_dump
Block dump from disk:

这样看来存储起来没有什么不一样。

推荐阅读:

ORA-01172、ORA-01151错误处理

ORA-00600 [2662]错误解决

ORA-01078 和 LRM-00109 报错解决方法

ORA-00471 处理方法笔记

ORA-00314,redolog 损坏,或丢失处理方法

ORA-00257 归档日志过大导致无法存储的解决办法

linux

Statement of this Website
The content of this article is voluntarily contributed by netizens, and the copyright belongs to the original author. This site does not assume corresponding legal responsibility. If you find any content suspected of plagiarism or infringement, please contact admin@php.cn

Hot AI Tools

Undresser.AI Undress

Undresser.AI Undress

AI-powered app for creating realistic nude photos

AI Clothes Remover

AI Clothes Remover

Online AI tool for removing clothes from photos.

Undress AI Tool

Undress AI Tool

Undress images for free

Clothoff.io

Clothoff.io

AI clothes remover

AI Hentai Generator

AI Hentai Generator

Generate AI Hentai for free.

Hot Article

Repo: How To Revive Teammates
1 months ago By 尊渡假赌尊渡假赌尊渡假赌
R.E.P.O. Energy Crystals Explained and What They Do (Yellow Crystal)
2 weeks ago By 尊渡假赌尊渡假赌尊渡假赌
Hello Kitty Island Adventure: How To Get Giant Seeds
1 months ago By 尊渡假赌尊渡假赌尊渡假赌

Hot Tools

Notepad++7.3.1

Notepad++7.3.1

Easy-to-use and free code editor

SublimeText3 Chinese version

SublimeText3 Chinese version

Chinese version, very easy to use

Zend Studio 13.0.1

Zend Studio 13.0.1

Powerful PHP integrated development environment

Dreamweaver CS6

Dreamweaver CS6

Visual web development tools

SublimeText3 Mac version

SublimeText3 Mac version

God-level code editing software (SublimeText3)

How does Go language implement the addition, deletion, modification and query operations of the database? How does Go language implement the addition, deletion, modification and query operations of the database? Mar 27, 2024 pm 09:39 PM

Go language is an efficient, concise and easy-to-learn programming language. It is favored by developers because of its advantages in concurrent programming and network programming. In actual development, database operations are an indispensable part. This article will introduce how to use Go language to implement database addition, deletion, modification and query operations. In Go language, we usually use third-party libraries to operate databases, such as commonly used sql packages, gorm, etc. Here we take the sql package as an example to introduce how to implement the addition, deletion, modification and query operations of the database. Assume we are using a MySQL database.

How does Hibernate implement polymorphic mapping? How does Hibernate implement polymorphic mapping? Apr 17, 2024 pm 12:09 PM

Hibernate polymorphic mapping can map inherited classes to the database and provides the following mapping types: joined-subclass: Create a separate table for the subclass, including all columns of the parent class. table-per-class: Create a separate table for subclasses, containing only subclass-specific columns. union-subclass: similar to joined-subclass, but the parent class table unions all subclass columns.

iOS 18 adds a new 'Recovered' album function to retrieve lost or damaged photos iOS 18 adds a new 'Recovered' album function to retrieve lost or damaged photos Jul 18, 2024 am 05:48 AM

Apple's latest releases of iOS18, iPadOS18 and macOS Sequoia systems have added an important feature to the Photos application, designed to help users easily recover photos and videos lost or damaged due to various reasons. The new feature introduces an album called "Recovered" in the Tools section of the Photos app that will automatically appear when a user has pictures or videos on their device that are not part of their photo library. The emergence of the "Recovered" album provides a solution for photos and videos lost due to database corruption, the camera application not saving to the photo library correctly, or a third-party application managing the photo library. Users only need a few simple steps

Detailed tutorial on establishing a database connection using MySQLi in PHP Detailed tutorial on establishing a database connection using MySQLi in PHP Jun 04, 2024 pm 01:42 PM

How to use MySQLi to establish a database connection in PHP: Include MySQLi extension (require_once) Create connection function (functionconnect_to_db) Call connection function ($conn=connect_to_db()) Execute query ($result=$conn->query()) Close connection ( $conn->close())

An in-depth analysis of how HTML reads the database An in-depth analysis of how HTML reads the database Apr 09, 2024 pm 12:36 PM

HTML cannot read the database directly, but it can be achieved through JavaScript and AJAX. The steps include establishing a database connection, sending a query, processing the response, and updating the page. This article provides a practical example of using JavaScript, AJAX and PHP to read data from a MySQL database, showing how to dynamically display query results in an HTML page. This example uses XMLHttpRequest to establish a database connection, send a query and process the response, thereby filling data into page elements and realizing the function of HTML reading the database.

Analysis of the basic principles of MySQL database management system Analysis of the basic principles of MySQL database management system Mar 25, 2024 pm 12:42 PM

Analysis of the basic principles of the MySQL database management system MySQL is a commonly used relational database management system that uses structured query language (SQL) for data storage and management. This article will introduce the basic principles of the MySQL database management system, including database creation, data table design, data addition, deletion, modification, and other operations, and provide specific code examples. 1. Database Creation In MySQL, you first need to create a database instance to store data. The following code can create a file named "my

How to handle database connection errors in PHP How to handle database connection errors in PHP Jun 05, 2024 pm 02:16 PM

To handle database connection errors in PHP, you can use the following steps: Use mysqli_connect_errno() to obtain the error code. Use mysqli_connect_error() to get the error message. By capturing and logging these error messages, database connection issues can be easily identified and resolved, ensuring the smooth running of your application.

Tips and practices for handling Chinese garbled characters in databases with PHP Tips and practices for handling Chinese garbled characters in databases with PHP Mar 27, 2024 pm 05:21 PM

PHP is a back-end programming language widely used in website development. It has powerful database operation functions and is often used to interact with databases such as MySQL. However, due to the complexity of Chinese character encoding, problems often arise when dealing with Chinese garbled characters in the database. This article will introduce the skills and practices of PHP in handling Chinese garbled characters in databases, including common causes of garbled characters, solutions and specific code examples. Common reasons for garbled characters are incorrect database character set settings: the correct character set needs to be selected when creating the database, such as utf8 or u

See all articles